:100000000C947C000C949B000C949B000C949B0023
:100010000C949B000C949B000C949B000C949B00F4
:100020000C949B000C94D80E0C949B000C949B0099
:100030000C949B000C949B000C949B000C949B00D4
:100040000C949B000C949B000C949B000C949B00C4
:100050000C949B000C949B000C949B000C949B00B4
:100060000C949B000C949B000C949B000C949B00A4
:100070000C949B000C949B000C9441040C949B00EA
:100080000C9404040C94E5040C949B00260F340F8C
:10009000550F650F700F840F900FB10FBC0FC90F74
:1000A000E60F0310480FF30F121027103F104A10ED
:1000B0006D10781083108F109C109E10AA10B6102F
:1000C0000F14141F14141700010E1315190E10002D
:1000D000040A040E111F110000001A050F140F006E
:1000E00000020E15150E0800040A0E010F110F0074
:1000F0000C12120C0000000011241FBECFEFD0E143
:10010000DEBFCDBF11E0A0E0B1E0E8E3F5E200E042
:100110000BBF02C007900D92AC39B107D9F715E0BB
:10012000ACE9B1E001C01D92A932B107E1F70E942C
:10013000B4000C949A120C9400001092620008957E
:10014000EF920F931F9386E9E82E01E010E021E083
:1001500040E050E060E070E087E491E00E940C072E
:100160001F910F91EF900895EF920F931F93F894C2
:100170000E946F090E94D10E0E94FE0C0E94A303F0
:100180000E949C0A81E08093080460E070E080E0B7
:1001900090E00E94C70478948FEF80936100809371
:1001A000620032E3E32E02E310E021E040E050E0A1
:1001B00060E070E08EE99AE00E940C0726E9E22EEA
:1001C00004EF11E021E040E050E060E070E084E8FE
:1001D00099E00E940C0700E117E221E040E050E0C6
:1001E00060E070E087E79EE00E940C0792E3E92E52
:1001F00000E513EC21E040E050E060E070E081E5D4
:100200009EE00E940C0708E91AE320E040E050E07D
:1002100060E070E080EC9EE00E940C070E941608EF
:10022000FDCFDF93CF930F92CDB7DEB780E4898304
:1002300041E0BE016F5F7F4F88E00E94BC060F90D7
:10024000CF91DF910895F8942091230530912405F2
:10025000409125055091260580910C0590910D0542
:10026000A0910E05B0910F05281739074A075B07C3
:1002700060F0789441E06EE971E082E00E94BC0693
:1002800083E291E00E945109089578940895DF93E4
:10029000CF93CDB7DEB760970FB6F894DEBF0FBE31
:1002A000CDBF81E0898342E0BE016F5F7F4F8DE06B
:1002B0000E94BC06882321F487E491E00E94510942
:1002C00060960FB6F894DEBF0FBECDBFCF91DF9121
:1002D0000895FC0180B1809580936200838982300B
:1002E00009F069C080919C0190919D0101969093C5
:1002F0009D0180939C0182818F3009F453C080312D
:1003000030F4833081F0843009F055C008C0803566
:1003100019F1853AE1F1803409F04DC008C08381BC
:10032000809310052DC083818093110529C02381FE
:100330003481922F80E0830F911D90931905809353
:10034000180525813681922F80E0830F911D9093AF
:10035000170580931605089521853285922F80E038
:10036000830F911D90931F0580931E052581368173
:10037000922F80E0830F911D90931D0580931C05A3
:1003800060E070E08DEF9EE00E94A80808958481EF
:100390009381382F20E0290F311D309321052093C0
:1003A0002005089583818093220568E873E18DEF2D
:1003B0009EE00E94A8080895EF92FF920F931F936A
:1003C000DF93CF9300D00F92CDB7DEB79C018C01A5
:1003D000FC019081923131F4809107058F5F809309
:1003E0000705A3C19131A1F4D90126EF34E0FD0145
:1003F0008181F9018083FD018181882309F495C100
:1004000011962F5F3F4FF5E026303F0781F78DC1F2
:10041000913009F08AC1F901F180F2E1FF1639F457
:1004200090939F01F092A00180910705CAC088E8CF
:10043000F816C1F48DEF9EE00E94510962E3E62EAA
:1004400000E61AEE21E040E050E060E070E08DEF61
:100450009EE00E940C0760E070E08DEF9EE00E943D
:10046000A80863C1E0EAFE1609F045C090939F0119
:10047000F092A001809103048093A1018091D9039F
:100480008093A2018091D903883119F48091EE0301
:1004900002C0809106048093A3018091040490918E
:1004A00005049093A4018091040490910504809325
:1004B000A50190919C0180919D018093A60190934C
:1004C000A701809107048093A8018091EE0390E03A
:1004D000959587958093A9018091EF038093AA0158
:1004E0008091DC038093AB018091DB038093AC01AE
:1004F0006EE070E016C1F3E1FF16B9F490939F012E
:10050000F092A001F894809126058093A10180913A
:1005100025058093A201809124058093A3018091F9
:1005200023058093A40178949FC084E1F816A9F470
:1005300090939F01F092A00180910F058093A101FB
:1005400080910E058093A20180910D058093A301F7
:1005500080910C058093A40187C0E0E3FE1679F436
:10056000F9828FEF8A8342E0BE016F5F7F4F87E0A1
:100570009B830E94BC069B8190939F01C3C0F1E2C4
:10058000FF1671F40D5F1F4FB801C80101970E945B
:10059000A40D81E080939F0181E28093A001B4C00B
:1005A00083E2F81689F481E080939F01F092A00124
:1005B000F9018281882319F48091110502C080918C
:1005C00010058093A101ABC0F2E2FF1641F40D5F6C
:1005D0001F4FB801C80101970E94540D90C080E9D7
:1005E000F816A9F4F89417BE15BC1EBC1FBC60E039
:1005F00070E080E090E00E94510E2DE088E190E0F4
:100600000FB6F894A89581BD0FBE21BDFFCFE0E4E1
:10061000FE1691F481E080939F01F092A0019091E9
:100620001805809119058093A1019093A2019091E2
:1006300016058091170514C0F0E5FF16C1F481E09E
:1006400080939F01F092A00190911C0580911D055F
:100650008093A1019093A20190911E0580911F05A6
:100660008093A3019093A40166E070E05AC081E5F5
:10067000F81641F40D5F1F4FB801C80101970E94A1
:10068000820D3DC0E2E5FE16A1F481E080939F015A
:10069000F092A001F90182818093A1016281E62F8D
:1006A000F0E0E65EFA4F80818093A20164E070E0A2
:1006B00038C0F0E7FF1699F481E080939F01F09233
:1006C000A00162E070E08FE991E00E94B4036DE068
:1006D00070E0F801828190E00E94150E26C0F0E6DD
:1006E000FF16A9F446E9E42E01E010E021E040E025
:1006F00050E060E070E087E491E00E940C0781E048
:1007000080939F01F092A00162E070E00AC081E056
:1007100080939F018FEF8093A0011092A10163E06D
:1007200070E08FE991E00E94B40380B180958093DE
:1007300062000F900F900F90CF91DF911F910F915A
:10074000FF90EF9008951092980083E080939900B5
:10075000EBE9F0E080818D7F808388ED80939A00C3
:1007600086E080939D000895AC0180919B0085FFF9
:10077000FCCF70939C006093C3021092D20310923E
:10078000D1036F5F7F4F7093D6036093D5036150A1
:10079000704081E090E09093D4038093D303DA011A
:1007A00020E030E007C02F5F3F4F8D91F901ED53FE
:1007B000FD4F808326173707B0F30895BC01809161
:1007C0009B0087FFFCCF30919C0080919B0087FFAE
:1007D000FCCF20919C00932F80E0AC01420F511D73
:1007E00020E030E00CC080919B0087FFFCCF80911F
:1007F0009C00FB01E20FF31F80832F5F3F4F241704
:10080000350788F3CA0108951F920F920FB60F9211
:100810000BB60F9211242F933F938F939F93EF93D7
:10082000FF932091D1033091D2038091D503909111
:10083000D6032817390780F48091D1039091D20311
:10084000FC01ED53FD4F208120939C000196909375
:10085000D2038093D10308C01092D2031092D10327
:100860001092D4031092D303FF91EF919F918F9137
:100870003F912F910F900BBE0F900FBE0F901F90C6
:1008800018951F920F920FB60F920BB60F9211246C
:10089000EF920F931F932F933F934F935F936F9319
:1008A0007F938F939F93AF93BF93EF93FF93809129
:1008B000C1029091C202892B99F481E090E090935B
:1008C000C2028093C10220919C00922F80E09093FD
:1008D000C0028093BF021092BE021092BD0241C0BE
:1008E0008091BD029091BE02892B69F48091BF0274
:1008F0009091C00220919C00820F911D9093C002A4
:100900008093BF0225C0E091BD02F091BE028091AC
:100910009C00E255FE4F80832091BD023091BE02C3
:100920008091BF029091C0022817390788F0109279
:10093000C2021092C102EE2400E010E020E04FEB72
:1009400052E06FEA71E08CED91E00E94940709C0DB
:100950008091BD029091BE0201969093BE02809359
:10096000BD02FF91EF91BF91AF919F918F917F91C8
:100970006F915F914F913F912F911F910F91EF9048
:100980000F900BBE0F900FBE0F901F901895809187
:100990000804880F81608093720080E48093700067
:1009A000E1E7F0E080818C7F80839FEF909373007C
:1009B00085ED8093740081E08093D9031092D80371
:1009C000909302041092ED0308951F920F920FB6B8
:1009D0000F920BB60F921124EF920F931F932F9348
:1009E0003F934F935F936F937F938F939F93AF93B7
:1009F000BF93EF93FF938091D903817C09F4B4C036
:100A00008091710090E0887F90708038910561F14D
:100A100081389105ACF48836910509F47BC089369C
:100A200091052CF48036910509F09CC089C080376F
:100A3000910509F485C08837910509F093C06AC013
:100A40008039910589F0813991052CF48838910518
:100A500009F088C082C08839910509F47EC0803AC7
:100A6000910509F07FC07CC08091D903803469F47E
:100A7000809173008093DB038FEF8093020480E802
:100A80008093D9031092D8036BC08091D90380382A
:100A900009F066C09091D8038091DB039817A0F409
:100AA0008091D803E82FF0E090917300E652FC4F5C
:100AB00092838F5F8093D80390910204809173009A
:100AC0008927809302044CC08091D8038031E1F4DF
:100AD000809173008093EC03909102048091EC0369
:100AE000981711F081E001C082E08093ED03EE24BD
:100AF00000E010E020E040E050E06AED73E089E6BD
:100B000091E00E94940729C08091D8038F5F809361
:100B1000D80326C0809106048F5F809306048091DD
:100B200003048A3068F422E3E22E02E310E020E0BE
:100B300040E050E060E070E08BE896E00E949407AF
:100B4000809173008093DA031092ED031092D80322
:100B500085EC8093740080E475C081E08093D903B4
:100B600085ECC1C085E4BFC08091710090E0887FB2
:100B700090708032910509F490C08132910554F44F
:100B80008031910599F088319105C9F0089709F0F5
:100B9000A6C00CC08033910509F457C08833910575
:100BA00009F459C0889709F09AC010C08091EE03EB
:100BB0008093730085E88093740088E043C01092AE
:100BC000D7038091EF038093730038C08091D703DF
:100BD0008131C1F485E98093740080E28093D90368
:100BE000109203048091040490910504019690935F
:100BF00005048093040460E070E087EC94E00E94B8
:100C0000E60873C09091D7038091EF03981750F0D6
:100C100080910004809373008091D7038F5F80934D
:100C2000D7030CC09091D703E92FF0E0E251FC4FBD
:100C30008281809373009F5F9093D70385E88093B0
:100C4000740080E18093D90350C0809106048F5FC7
:100C50008093060427C0809106048F5F809306046A
:100C600060E070E087EC94E00E94E6088091030465
:100C70008A3070F492E3E92E02E310E020E040E0D5
:100C800050E060E070E08BE896E00E94940703C0BB
:100C900088E28093D90385E826C0809107048F5F9E
:100CA0008093070460E070E087EC94E00E94E6081F
:100CB000809103048A3070F482E3E82E02E310E0AE
:100CC00020E040E050E060E070E08BE896E00E94B9
:100CD000940703C088E28093D90385E904C084E0C7
:100CE0008093D90385E080937400FF91EF91BF91C9
:100CF000AF919F918F917F916F915F914F913F91B4
:100D00002F911F910F91EF900F900BBE0F900FBE80
:100D10000F901F901895EF920F931F938091D90316
:100D2000813061F042E3E42E05E010E020E040E095
:100D300050E060E070E08BE896E018C01092D703B6
:100D400085EA8093740082E08093D9038091030444
:100D50008F5F8093030432E3E32E04EF11E020E081
:100D600040E050E060E070E087EC94E00E940C0707
:100D70001F910F91EF900895EF920F931F93582FAB
:100D800080910304882309F441C0809103048A30D0
:100D9000E9F181E037C08FEF80930004DB0120E0B0
:100DA00030E00DC08C91F901E251FC4F82838091BB
:100DB00000049D918927809300042F5F3F4F2417E3
:100DC00088F381E080930304852F90E0880F991FBA
:100DD0008093EE034093EF031092D70385EA80934C
:100DE000740082E08093D90352E3E52E04EF11E012
:100DF00020E040E050E060E070E087EC94E00E948A
:100E00000C0780E01F910F91EF9008958091D90316
:100E1000813009F282E0F6CFCF92DF92EF92FF921B
:100E20000F931F93CF93DF936C01F22E9E2D20E042
:100E300030E0A22FF901B4E0EE0FFF1FBA95E1F701
:100E4000E75FFB4F8685882331F0AF5F2F5F3F4F11
:100E50002C30310571F7CA2FD0E0DE0124E0AA0F53
:100E6000BB1F2A95E1F7A75FBB4F1196DC92CE928C
:100E7000FE0184E0EE0FFF1F8A95E1F7E55FFB4F6F
:100E800071836083FE0164E0EE0FFF1F6A95E1F756
:100E9000E35FFB4F51834083FD01F682992311F4F8
:100EA000178607C0923311F481E001C082E0FD0192
:100EB000878734E0CC0FDD1F3A95E1F7DE01A75FAD
:100EC000BB4FFD018785282F30E027533B4FF901A9
:100ED0008081980FFD0195878F5FF9018083FD0167
:100EE0001087078381E08687F8942091230530914D
:100EF00024054091250550912605C801A0E0B0E0E9
:100F0000820F931FA41FB51FC75FDB4F89879A8786
:100F1000AB87BC877894DF91CF911F910F91FF90A1
:100F2000EF90DF90CF900895CF92DF92EF92FF92F3
:100F30000F931F93CF93DF93EC016B01F22E9E2D45
:100F400020E030E0E22EF901A4E0EE0FFF1FAA95A9
:100F5000E1F7E75FFB4F8685882331F0E3942F5F4D
:100F60003F4F2C30310571F76E2D70E0DB01E4E06E
:100F7000AA0FBB1FEA95E1F7A75FBB4F1196DC9361
:100F8000CE93FB0134E0EE0FFF1F3A95E1F7E55FEA
:100F9000FB4FD182C082FB0124E0EE0FFF1F2A9598
:100FA000E1F7E35FFB4F51834083ED01FE8299231C
:100FB00011F41F8609C0923321F481E0FD01878777
:100FC00003C082E0ED018F8784E0660F771F8A956A
:100FD000E1F7675F7B4FEB01EF85F0E0E753FB4FF5
:100FE0008081980F9D878F5F808318870F8381E0B2
:100FF0008E8720912305309124054091250550913D
:101000002605C801A0E0B0E0820F931FA41FB51F02
:10101000FB0181879287A387B487DF91CF911F91CE
:101020000F91FF90EF90DF90CF900895CF93DF93D3
:10103000F894409123055091240560912505709105
:10104000260578941092CC048091CF048F5F809312
:10105000CF048091CF04883C49F48091CE048695DA
:101060008093CD041092CE041092CF04EFEFFFEFE7
:1010700020E030E0E901A4E0CC0FDD1FAA95E1F704
:10108000C75FDB4F8E85882399F08091CC048F5FFA
:101090008093CC0489859A85AB85BC854817590710
:1010A0006A077B0728F08D858F1710F4FD85E22FE6
:1010B0002F5F3F4F2C303105E9F6EF3F09F444C074
:1010C0008091CE048F5F8093CE04FF27E7FDF095DB
:1010D00094E0EE0FFF1F9A95E1F7EF01C75FDB4F3A
:1010E00028813981DF01A35FBB4F6D917C91E55F62
:1010F000FB4F80819181F90109958E81882349F404
:101100001E86EF85F0E0E753FB4F8081815080839E
:101110001BC08E81833011F481E004C08E81823047
:1011200019F483E08E8310C029853A854B855C8550
:101130008F819885A0E0B0E0820F931FA41FB51F98
:1011400089879A87AB87BC8781E0DF91CF9108952B
:10115000CF93DF939C01E0E0F0E0DF0144E0AA0FD1
:10116000BB1F4A95E1F7A75FBB4F8D919C911197EB
:101170008217930721F5ED018E85882301F18E8179
:10118000833009F1F8942091230530912405409192
:10119000250550912605CB01A0E0B0E0820F931FFA
:1011A000A41FB51F24E0EE0FFF1F2A95E1F7E75FAC
:1011B000FB4F81879287A387B487789404C03196C8
:1011C000EC30F10551F6DF91CF910895AC0120E0AC
:1011D00030E0F901A4E0EE0FFF1FAA95E1F7E75F09
:1011E000FB4F8081918184179507B9F48685882308
:1011F000A1F02091230530912405409125055091BF
:101200002605CB01A0E0B0E0820F931FA41FB51FFD
:1012100081879287A387B48708952F5F3F4F2C3033
:101220003105B9F60895CF93DF939C01C0E0D0E07B
:10123000FE0144E0EE0FFF1F4A95E1F7E75FFB4F29
:10124000808191818217930729F58685882311F182
:10125000F894209123053091240540912505509163
:101260002605CB01A0E0B0E0820F931FA41FB51F9D
:1012700024E0CC0FDD1F2A95E1F7FE01E75FFB4F6D
:1012800081879287A387B4877894C75FDB4F82E01A
:101290008E8304C02196CC30D10551F6DF91CF91D9
:1012A0000895AC0120E030E0F90164E0EE0FFF1F8B
:1012B0006A95E1F7E75FFB4F80819181841795077D
:1012C00041F41686E785F0E0E753FB4F80818150BB
:1012D00080832F5F3F4F2C30310531F7089580E038
:1012E00090E0FC0174E0EE0FFF1F7A95E1F7E75FF5
:1012F000FB4F168601968C30910599F7089560E0B2
:1013000080680E94FC0B089560E081E00E94FC0B65
:1013100080E00E947F098091E104843009F490C04C
:10132000853058F4813051F18130D0F0823009F4A9
:101330005BC0833009F0FFC079C0873009F4BDC0BD
:10134000883038F4853009F485C0863009F0F3C060
:1013500099C0883009F4CCC0893009F0ECC0D5C000
:1013600086EF94E00E94DF0C80E40E947F0980E019
:1013700091E00E94DF0C6091070534C086E091E0A7
:101380000E94DF0C8091D903883189F480E40E94A7
:101390007F096091EE0370E075956795882777FD6A
:1013A0008095982F0E94380C80E191E03CC06091BC
:1013B000D90370E080E090E00E94380C86E191E073
:1013C0000E94DF0C6091060470E080E090E00E94D3
:1013D000380C80E40E947F0988E191E00E94DF0CD4
:1013E0006091030470E08CC085E291E00E94DF0C04
:1013F0006091CC0470E080E090E00E94380C8EE2B6
:1014000091E00E94DF0C80E40E947F0982E391E07A
:101410000E94DF0C6091CD0470E080E090E00E94BB
:10142000380C8DE391E00E94DF0C08958FE391E08A
:101430000E94DF0C80E40E947F0960911005D2CFEA
:101440008DE491E00E94DF0C80E40E947F096091AE
:101450001105C8CF88E591E00E94DF0C6091180566
:101460007091190580E090E00E94380C80E40E94A1
:101470007F0980E691E00E94DF0C60911605709173
:1014800017053EC087E691E00E94DF0C60911A05C7
:1014900070E080E090E00E94380C8DE391E00E94C3
:1014A000DF0C80E40E947F0981E791E00E94DF0C5D
:1014B00060911C0570911D0523C08BE791E00E948F
:1014C000DF0C60911B0570E080E090E00E94380C1A
:1014D0008DE391E00E94DF0C80E40E947F0981E7A8
:1014E00091E00E94DF0C60911E0570911F0508C0FD
:1014F00085E891E00E94DF0C6091990170919A015A
:1015000080E090E00E94380C08958DE891E00E9400
:10151000DF0C609120057091210580E090E00E9431
:10152000380C80E40E947F096091220570E080E021
:1015300090E00E94380C08951ABA0895EF920F9324
:101540001F93CF93DF93A2EEB4E0CCEED4E050E053
:1015500020E030E061E04C91F901E951FB4F40831C
:10156000188289B390E0022E02C0959587950A945F
:10157000E2F780FF02C06C9305C01C92413011F469
:10158000488351E02F5F3F4F11962196253031055A
:1015900011F7513061F4EE2400E010E020E040E06B
:1015A00050E060E070E08DED9AE00E940C07DF9162
:1015B000CF911F910F91EF900895EF920F931F938A
:1015C000DF93CF9300D00F92CDB7DEB78091EE04BA
:1015D000813009F04AC08091E104833051F4809158
:1015E00010058F5F8983853008F0198281E08A8336
:1015F0000AC0843081F4809111058F5F8983853022
:1016000008F019821A82BE016F5F7F4FCE010296E9
:101610000E94A40DBEC0882369F4EE2400E010E00F
:1016200020E040E050E060E070E080EC9EE00E944E
:101630000C07AFC0853041F480E48B8341E0BE01EC
:101640006D5F7F4F88E00EC0863011F48FE004C0DC
:10165000873009F09EC080EF8B8341E0BE016D5F53
:101660007F4F8CE00E94BC0694C08091ED048130D5
:1016700051F48091E104882311F489E001C0815084
:101680008093E10486C08091F004813049F4809118
:10169000E104893019F41092E1047BC08F5FF0CF30
:1016A0008091EC04813079F58091E104863059F421
:1016B00080911A058B5F80931A058436B0F184E619
:1016C00080931A0532C0873059F480911B058B5FD7
:1016D00080931B058536C0F184E680931B0534C0DA
:1016E000883009F056C08091990190919A01C29674
:1016F00090939A0180939901855A964008F441C0CD
:1017000084EA96E03AC08091EF04813009F041C04C
:101710008091E104863069F480911A0585508093A8
:101720001A05843610F010921A051A826AE175E0E3
:101730000FC0873091F480911B05855080931B0565
:10174000843610F010921B0581E08A836BE175E00E
:10175000CE0102960E94820D1CC08830D1F4809187
:10176000990190919A01C29790939A01809399015F
:101770008C5B924030F48CEB92E090939A018093D2
:10178000990183E08A8369E971E0CE0102960E94A3
:10179000540D82E3E82E00E010E020E040E050E04D
:1017A00060E070E084E899E00E940C070F900F90D1
:1017B0000F90CF91DF911F910F91EF90089587E0E7
:1017C00084BB8AE780F985BB000090E022E0AA9AFA
:1017D0009295000000000000000083B3AA9883FDEA
:1017E000916084FD926085FD946086FD9860215033
:1017F00071F715BA892F08950F931F93CF93DF9335
:10180000182F062F15BA8091F104882361F1E8940E
:10181000C0E0D0E00E94DF0B87FF21C0219683E06B
:10182000C83ED807B9F71092F1048FE784BB22E0D5
:10183000802F011181E0912F14FD886095FD80615A
:1018400096FD806217FD806485BB0000AA9A129500
:1018500000000000000085BB215051F704C0C85EA5
:10186000D3401CF3E0CFDF91CF911F910F910895EA
:101870009F92AF92BF92CF92DF92EF92FF920F931F
:101880001F93CF93DF937B018C0197FF0BC01095C3
:101890000095F094E094E11CF11C011D111D61E024
:1018A0008DE207C0611571058105910521F461E0A4
:1018B00080E30E94FC0BA12C8AECB82E8AE9C82E8A
:1018C0008BE3D82E9924CAE0D0E0C801B701A60165
:1018D00095010E947F12992011F4222391F061E07A
:1018E000822F805D0E94FC0BC801B701A601950103
:1018F0000E947F12AC01CB01DA017C018D01992499
:101900009A94C601B5012AE030E040E050E00E9420
:101910007F12C901DA015C016D012197B1F6DF91F7
:10192000CF911F910F91FF90EF90DF90CF90BF90DC
:10193000AF909F900895AF92BF92CF92DF92EF92B7
:10194000FF920F931F937B018C015A01CC24DD245D
:10195000C601B5010E946C119B01AC01C801B70121
:101960000E94FA110E943B117B018C01C801A60163
:1019700095010E947F12CA01B9010E94380C61E0F2
:101980008EE20E94FC0BB701C801A60195010E94DE
:101990007F120E946E119F7720E030E040E05FE30D
:1019A0000E94D7100E943B110E94380C1F910F918A
:1019B000FF90EF90DF90CF90BF90AF900895CF93BE
:1019C000DF93EC0104C0219661E00E94FC0B88814A
:1019D0008823C9F7DF91CF910895CF93DF93FC015E
:1019E000EC01849105C061E00E94FC0BFE01849132
:1019F00021968823C1F7DF91CF9108950F931F930C
:101A000081E08093F1048FE784BB4FE024E030E075
:101A10006FEF7FE350E1CB010197F1F741FB83F9D1
:101A200085BB0000AA9A0000000000000000AA98F0
:101A300046952150304079F760E088E20E94FC0B27
:101A40008091F104882319F160E086E00E94FC0B8C
:101A500060E082E00E94FC0B60E08CE00E94FC0BE6
:101A600060E088E40E94FC0BE0ECF0E008C08F012D
:101A70000F5F1F4F849161E00E94FC0BF80180E032
:101A8000E83FF807A0F360E080E80E94FC0B80E0EC
:101A90001F910F910895E8940E94DF0B60E0806829
:101AA0000E94FC0B80E00895DF93CF9300D0CDB768
:101AB000DEB7FC014081FB013081842F90E0817012
:101AC000907024E0880F991F2A95E1F78071218199
:101AD0002F70822B89833A83423030F442E0BE017A
:101AE0006F5F7F4F83E007C0443038F442E0BE01AF
:101AF0006F5F7F4F84E00E94BC060F900F90CF91E4
:101B0000DF910895DF93CF9300D0CDB7DEB7FC010E
:101B1000DB01E0819C918E2F81708983953608F0DE
:101B200094E69A83F0E0E170F070E65EFA4F9083FD
:101B300042E0BE016F5F7F4F86E00E94BC060F90BF
:101B40000F90CF91DF910895DF93CF9300D000D015
:101B5000CDB7DEB7FC01E081DB0190E08C918330F2
:101B600009F491E099838C918350823010F081E0E8
:101B700001C082E0982B99831A828EE18B83EE2339
:101B800059F4906899838C918093110543E0BE01CC
:101B90006F5F7F4F83E040C0E13059F490689983D4
:101BA0008C918093100543E0BE016F5F7F4F84E00E
:101BB00033C08E2F8250823078F4E33011F4906875
:101BC0009983F0E0E05FFA4F8C91808343E0BE019F
:101BD0006F5F7F4F89E020C08E2F8450823078F471
:101BE000E53011F490689983F0E0E05FFA4F8C9152
:101BF000808343E0BE016F5F7F4F8AE00DC0E63017
:101C000069F48FE089838C918A838093220542E076
:101C1000BE016F5F7F4F8FE00E94BC060F900F9058
:101C20000F900F90CF91DF910895CF92DF92EF92B6
:101C30000F931F93DF93CF9300D0CDB7DEB76C0126
:101C40008B0181E0898391E0C916D10411F48A8364
:101C500008C06D30710521F485E19EE00E945109B4
:101C60001A8242E0BE016F5F7F4F802F0E94BC0648
:101C70000D30110561F432E3E32E04E610E020E0BC
:101C80004EE050E0B60185E19EE00E940C070F9007
:101C90000F90CF91DF911F910F91EF90DF90CF9038
:101CA0000895EF920F931F93DF93CF930F92CDB7C9
:101CB000DEB781E3898341E0BE016F5F7F4F87E03C
:101CC0000E94BC06882361F0EE2404EF11E020E0BE
:101CD00040E050E060E070E081E59EE00E940C078B
:101CE0000F90CF91DF911F910F91EF900895DF93A7
:101CF000CF9300D000D00F92CDB7DEB720910C0566
:101D000030910D0540910E0550910F0521153105BB
:101D100041055105B9F0F8946091230570912405AF
:101D20008091250590912605621B730B840B950B02
:101D3000789420E63AEE40E050E00E945D123A834B
:101D4000298304C08FEF9FEF9A838983FE01339626
:101D500083E0DF011D928A95E9F785E18B83898114
:101D60008C838A818D8363E070E0CF010E94B4038D
:101D70000F900F900F900F900F90CF91DF910895DB
:101D8000DF93CF930F92CDB7DEB784E3898361E011
:101D900070E0CE0101960E94B4030F90CF91DF91C5
:101DA00008958BE085BD89EF83BD80E887BF0895E6
:101DB0001F920F920FB60F9211248F939F93AF93A0
:101DC000BF938091230590912405A0912505B091A2
:101DD00026050196A11DB11D80932305909324052E
:101DE000A0932505B0932605BF91AF919F918F9148
:101DF0000F900FBE0F901F9018951F93DF93CF93F6
:101E0000CDB7DEB728970FB6F894DEBF0FBECDBFB3
:101E100021E0298384E08A832B8388E998E09887EE
:101E20008F832C8382E38D838FE08E8380912705BF
:101E3000E82FF0E0EA31F10508F0AEC1EA5BFF4FB0
:101E4000EE0FFF1F0590F491E02D099411E0198326
:101E500084E08A83BE016E5F7F4FCE0101960E94AF
:101E6000A40D1093270598C181E08B838091100504
:101E7000823009F091C188E998E098878F83BE018C
:101E8000695F7F4FCE0103960E94540D8CE07CC1A8
:101E900085E0898383E08A83BE016E5F7F4FCE0138
:101EA00001960E94A40D82E06FC113E01B8388E5B8
:101EB00092E098878F83BE01695F7F4FCE010396C2
:101EC0000E94540D1093270561C1198283E08A8313
:101ED000BE016E5F7F4FCE0101960E94A40D1EC011
:101EE00080911105813009F057C186E0898384E033
:101EF0008A83BE016E5F7F4FCE0101960E94A40DC2
:101F000085E0809327052AC0809122058130C9F0A1
:101F100060E177E28DEF9EE00E94130984E03EC00D
:101F200080912205823069F481E08C8382E38D8385
:101F3000BE016B5F7F4FCE0104960E94820D87E049
:101F400023C116E0198383E08A83BE016E5F7F4F51
:101F5000CE0101960E94A40D1093270560E177E25F
:101F600017C18FE08E8341E0BE016A5F7F4F8CE036
:101F70000E94BC0688E008C181E0898383E08A83EF
:101F8000BE016E5F7F4FCE0101960E94A40D89E0D5
:101F900059C080911005813021F48BE18093270591
:101FA000FBC080911E0590911F05843C910508F0AF
:101FB000F3C081E0898384E08A83BE016E5F7F4F36
:101FC000CE0101960E94A40D8AE03CC081E08C8382
:101FD00082E38D83BE016B5F7F4FCE0104960E942A
:101FE000820D8DE0D1C0198284E08A83BE016E5FCC
:101FF0007F4FCE0101960E94A40D8BE080932705B0
:1020000068E873E1C5C083E08B838CED95E0988729
:102010008F83BE01695F7F4FCE0103960E94540DEE
:102020008EE0B2C080911105823009F0B5C084E61F
:102030008D831C82BE016B5F7F4FCE0104960E9490
:10204000820D8FE08093270568EB7BE0A1C0809133
:102050001C0590911D058F55914008F09DC0198277
:1020600083E08A83BE016E5F7F4FCE0101960E949E
:10207000A40D80E18093270568E97AE389C019827D
:102080001A82BE016E5F7F4FCE0101960E94A40DA1
:1020900081E17AC094E0998380912805BE016E5F4A
:1020A0007F4F9E012F5F3F4F823078F49A83C901A2
:1020B0000E94A40D81E180932705809128058F5F00
:1020C0008093280560E375E763C0109228051A82A3
:1020D000C9010E94A40D82E157C080EF8E8341E0C8
:1020E000BE016A5F7F4F8CE00E94BC0683E14CC05A
:1020F0001C821D82BE016B5F7F4FCE0104960E9441
:10210000820D84E141C081E08C831D82BE016B5F42
:102110007F4FCE0104960E94820D85E135C081E09B
:10212000898384E08A83BE016E5F7F4FCE01019672
:102130000E94A40D86E128C087E126C06DE070E012
:1021400081E090E00E94150E88E18093270560E20F
:102150007EE41EC06DE070E080E090E00E94150E0D
:1021600089E18093270560ED77E012C081E08B83E1
:102170008CED95E098878F83BE01695F7F4FCE011C
:1021800003960E94540D8AE18093270568EC70E065
:102190008DEF9EE00E94130928960FB6F894DEBFDB
:1021A0000FBECDBFCF91DF911F9108955058BB272F
:1021B000AA270ED0E5C0D6D030F0DBD020F031F425
:1021C0009F3F11F41EF4CBC00EF4E095E7FBC1C0B5
:1021D000E92FE7D080F3BA176207730784079507E2
:1021E00018F071F49EF5FFC00EF4E0950B2EBA2F97
:1021F000A02D0B01B90190010C01CA01A00111240D
:10220000FF27591B99F0593F50F4503E68F11A16B8
:10221000F040A22F232F342F4427585FF3CF469549
:1022200037952795A795F0405395C9F77EF41F166B
:10223000BA0B620B730B840BBAF09150A1F0FF0F35
:10224000BB1F661F771F881FC2F70EC0BA0F621F21
:10225000731F841F48F4879577956795B795F79511
:102260009E3F08F0B3CF9395880F08F09927EE0FA3
:1022700097958795089504D06894B111B5C00895D5
:1022800098D088F09F5790F0B92F9927B751A0F0B8
:10229000D1F0660F771F881F991F1AF0BA95C9F7FA
:1022A00012C0B13081F09FD0B1E008959CC0672F7B
:1022B000782F8827B85F39F0B93FCCF386957795AA
:1022C0006795B395D9F73EF4909580957095619593
:1022D0007F4F8F4F9F4F0895E89409C097FB3EF4BE
:1022E00090958095709561957F4F8F4F9F4F992363
:1022F000A9F0F92F96E9BB279395F69587957795E1
:102300006795B795F111F8CFFAF4BB0F11F460FFA0
:102310001BC06F5F7F4F8F4F9F4F16C0882311F0F8
:1023200096E911C0772321F09EE8872F762F05C00C
:10233000662371F096E8862F70E060E02AF09A95A7
:10234000660F771F881FDAF7880F9695879597F99C
:10235000089597F99F6780E870E060E008959FEF27
:1023600080EC089500240A9416161706180609062C
:10237000089500240A9412161306140605060895FB
:10238000092E0394000C11F4882352F0BB0F40F483
:10239000BF2B11F460FF04C06F5F7F4F8F4F9F4FC3
:1023A000089557FD9058440F551F59F05F3F71F045
:1023B0004795880F97FB991F61F09F3F79F08795AC
:1023C0000895121613061406551FF2CF4695F1DF35
:1023D00008C0161617061806991FF1CF86957105C5
:1023E000610508940895E894BB2766277727CB01F9
:1023F00097F908950BD0C4CFB5DF28F0BADF18F0F5
:10240000952309F0A6CFABCF1124EECFCADFA0F3FE
:10241000959FD1F3950F50E0551F629FF001729F79
:10242000BB27F00DB11D639FAA27F00DB11DAA1F98
:10243000649F6627B00DA11D661F829F2227B00DE5
:10244000A11D621F739FB00DA11D621F839FA00D70
:10245000611D221F749F3327A00D611D231F849FC0
:10246000600D211D822F762F6A2F11249F57504017
:102470008AF0E1F088234AF0EE0FFF1FBB1F661FB2
:10248000771F881F91505040A9F79E3F510570F06B
:1024900060CFAACF5F3FECF3983EDCF3869577954B
:1024A0006795B795F795E7959F5FC1F7FE2B880F66
:1024B000911D9695879597F90895A1E21A2EAA1B6A
:1024C000BB1BFD010DC0AA1FBB1FEE1FFF1FA217E4
:1024D000B307E407F50720F0A21BB30BE40BF50BE1
:1024E000661F771F881F991F1A9469F7609570956A
:1024F000809590959B01AC01BD01CF01089597FB9C
:10250000092E05260ED057FD04D0D7DF0AD0001CB7
:1025100038F450954095309521953F4F4F4F5F4F80
:102520000895F6F790958095709561957F4F8F4F40
:082530009F4F0895F894FFCFBE
:10253800486974733A0054776920737461743A0077
:10254800204E41434B002F004E756D20726574720A
:102558006965733A004F5320696E666F3A002F31F0
:1025680032004350552075736167653A002500466F
:10257800696C746572206D6F746F723A0041726D88
:10258800206D6F746F723A00436F666665653A0036
:1025980057617465723A0056616375756D20313AFA
:1025A8000043757272656E743A20005661637575E2
:1025B8006D20323A00536572766F333A0041726D7E
:0C25C80020706572696F643A00E803003F
:00000001FF
